:020000020000FC
:100000007BC048C079C078C077C040C075C074C09C
:1000100073C072C071C070C06FC06EC06DC0D39429
:100020003D2D313208F0CC24CC2019F4C398C4986B
:100030000895332797FF02C0C39A01C0C398990F50
:1000400008F43FEFAA0F08F49160332309F0A16090
:100050003327B7FF02C0C49A01C0C498BB0F08F48D
:100060003FEFCC0F08F4B160332309F0C16008956D
:10007000E199FECF4EBB8DBBE29AE19A0895E199DA
:10008000FECF4EBBE09A5CB38DB30895FFB72395C6
:10009000FFBF1895DF93DFB7DF938394BB20B9F0E0
:1000A00062B7722F332732BF38BF2227DD24733C5B
:1000B00050F4763040F03FEFC32E9E2DAF2DB02F81
:1000C000C12FADDF04C0C398C498CC2400C0DF9119
:1000D000DFBFDF91189595E00FEF3FEF3A95F1F70D
:1000E0000A95D9F79A95C1F70895C39AC49AF3DF90
:1000F000C398C498F0DF08953FED3DBFC398C498FE
:10010000BB9ABC9ABA98C29A33273FBBEEDFBB2496
:100110008824882730E43BBF32E035BF222735E012
:1001200033BF32E039BF7894881510F4DEDF882DB4
:100130002839D0F3332733BF32BFF8948230F0F040
:100140008530E0F4D2DFD1DFD0DF88242227882772
:1001500035E033BF7894881528F4882D8E3021F04F
:100160002227C3DF2839B8F3332733BF32BF332701
:1001700035BFF89444277CDFB8DFB7DFB6DF44270C
:100180007EDF8823E1F08A95E1F08A95E1F08A9597
:10019000E1F08A95E1F08A95E1F08A95E1F08A959F
:1001A000E1F08A95E1F08A95E1F08A95E1F08A958F
:1001B000E1F08A95E1F08A95E1F04CE31CC044E05F
:1001C0001AC048E018C04CE016C040E114C044E139
:1001D00012C048E110C04CE10EC040E20CC044E245
:1001E0000AC048E208C04CE206C040E304C044E351
:1001F00002C048E300C043DFE82E439540DFF82EFD
:1002000043953DDF082F43953ADF182F33E033BF86
:1002100022273FEFB32ECC2432E039BF32E035BF86
:1002200078943D2D3130E9F7482DEFEF572F862F89
:100230006695769508F460686695769508F460682A
:100240006695769508F460686695769508F460681A
:100250006695769508F46068972EA62E752F682F00
:10026000552788273FE1532E8A0D591D481509F05F
:10027000D8CF2517D9F732B73817C0F3D0DE5A9444
:1002800099F78A0D591D481509F0CBCF2517D9F7D5
:0C02900032B73817C0F3C398C498C3CF2E
:00000001FF
